:101BDD005753746174696F6E000408000001503032
:101BED005431000000000101430408000001503091
:101BFD00543200000000010147040800000150307C
:101C0D0054330000000001014B0408000001503066
:101C1D0054340000000001014F0408000001503150
:101C2D00543500000000010153040800000150313B
:101C3D005436000000000101570408000001503126
:101C4D0054370000000001015B0408000001503111
:101C5D0054380000000001015F04080000015032FB
:101C6D0054300000000001016304080000015032EF
:101C7D00543100000000010167045A000001503288
:101C8D0052480000000001016B045A00000150325F
:101C9D004F320000000001016F04080000015033B5
:101CAD00543000000000010173040800000150339E
:101CBD00543100000000010177045A000001503337
:101CCD0052480000000001017B045A00000150330E
:101CDD004F320000000001017F00000000000000F5
:091CED00000000000000000000EE
:102A7F00011A01430183FF1BE6410140004201415E
:022A8F00000045
:0F2A95009001A0EFF0E4F5A775A45D75A5FF22F1
:0E2AC20090FFFF1210C5EFF09000010210C54A
:08000300900196EFF07F00224E
:10283900900196EBF0A3EAF0A3E9F0900196E0FB92
:10284900A3E0FAA3E0F9120E7CFF900199E0FBA343
:10285900E0FAA3E0F9EF120EC2900196E0FBA3E0C3
:10286900FAA3E0F9900001120E95FF900199E0FB9F
:10287900A3E0FAA3E0F9900001EF120ED47F02223F
:1011B400E49001A6F0122AD0C8ECC8C9EDC9CAEE61
:1011C400CACBEFCB900142E02414FF900141E034FC
:1011D40000FEE4FCFDC3120FC950037F0022122A53
:1011E400D0900141EEF0A3EFF0C280D282C2937F8F
:1011F400017E001225EC7F0112295E30810CD2930E
:101204007F017E001225EC7F0022900140E004540F
:101214000FFF540133333354F844B0FEEFC3134E7D
:1012240090019DF05480D394004003D38001C39275
:101234008290019DE0FF25E0F0E490019CF0900194
:101244009E12103E000000007F017E001225ECD2A9
:101254008090019EE0FCA3E0FDA3E0FEA3E0FF7804
:1012640001120FEEC8ECC8C9EDC9CAEECACBEFCB68
:10127400A281E4334BFFEAFEE9FDE8FC90019E12F3
:1012840010197F017E001225ECC28090019DE0FFC1
:101294005480D394004003D38001C39282EF25E0AD
:1012A40090019DF090019CE004F0E0C394184098F4
:1012B400D280D282D29390019EE0FCA3E0FDA3E011
:1012C400FEA3E0FF7814120FDAE47B03FAF9F8C303
:1012D400120FB3700C9001A212103E3FA0000080C8
:1012E4002190019EE0FCA3E0FDA3E0FEA3E0FF78D3
:1012F40014120FDAEC4D4E4F7011A312103EBFA022
:1013040000009001A67401F002139790019EE0FC86
:10131400A3E0FDA3E0FEA3E0FF7815120FDAE47B5F
:1013240001FAF9F8C3120FB390019E7010A3E0FD07
:10133400A3E0FEA3E0FFED540FFDE4800FA3E0FD66
:10134400A3E0FEA3E0FFED44F0FD74FFFC90019EDA
:1013540012101990019EE0FCA3E0FDA3E0FEA3E0BF
:10136400FFEC120DBD9001A2121019E4FBFA798072
:1013740078499001A2E0FCA3E0FDA3E0FEA3E0FF16
:10138400120CA7E4FBFA79A0783F120B9E9001A2FD
:101394001210197B007A40791C78459001A2E0FC78
:1013A400A3E0FDA3E0FEA3E0FF120CA77B007A24D8
:1013B40079747849120B9E9001A212101990014081
:1013C400E05403600A64016006E0C39408503F904F
:1013D40001A2E0FCA3E0FDA3E0FEA3E0FF7B9A7A78
:1013E40099798878C3120AAD9001A2121019E4FF0A
:1013F400FE7DC87CC29001A2E0F8A3E0F9A3E0FA64
:10140400A3E0FB120D4440030214D40214CA900159
:1014140040E05403FFBF02487F907EB57DE07CBD71
:101424009001A2E0F8A3E0F9A3E0FAA3E0FB120B19
:101434009E7BD07AA379D47842120AAD9001A2128D
:101444001019E4FFFE7DC87C429001A2E0F8A3E0FD
:10145400F9A3E0FAA3E0FB120D44607440728066C5
:10146400E4FFFE7D487CC39001A2E0F8A3E0F9A369
:10147400E0FAA3E0FB120AADE4FBFA7948784312E0
:101484000CA7E4FBFA79C87842120B9E9001A212D1
:101494001019E4FFFEFDFC9001A2E0F8A3E0F9A31B
:1014A400E0FAA3E0FB120D44401CE4FFFE7DF07C57
:1014B400419001A2E0F8A3E0F9A3E0FAA3E0FB1253
:1014C4000D44600C400A9001A212103EC2C80000F4
:1014D400E4FFFE7D7A7C449001A2E0F8A3E0F9A346
:1014E400E0FAA3E0FB120B9EE4FBFAF9783F120A40
:1014F400AD121E00E4FBFA797A7844120CA790012D
:10150400A21210199001A6E0B4010A9001A21210CF
:101514003EC2CA00009001A2E0FCA3E0FDA3E0FEED
:10152400A3E0FF900140E0FB25E025E02443F582A1
:10153400E43401F583121019EB04540F900140F0C8
:021544007F0125
:011546002282
:032AEE000211B41E
:10000E00323032322D30372D3132202D20313233F5
:05001E00343536370007
:10197E007BFF7A00790E7D2D122572EA494B601F8E
:10198E007BFF7A00790E7D2D122572E92402F9E48F
:10199E003AFA9001A0EBF0A3EAF0A3E9F08004E498
:1019AE00FEFF229001A0E0FBA3E0FAA3E0F9900075
:1019BE0001120E95FFC39430400CEFD394395006AC
:1019CE00EF24D0FF801A900001120E95FFC3946190
:1019DE00400CEFD394665006EF24A9FF80027F00DF
:1019EE00EF7D00FC120E7CFFC39430400CEFD394BD
:1019FE00395006EF24D0FF80229001A0E0FBA3E037
:101A0E00FAA3E0F9120E7CFFC39461400CEFD3945D
:101A1E00665006EF24A9FF80027F00EFC454F04CFD
:101A2E00FC9001A0E0FBA3E0FAA3E0F99000021203
:101A3E000E95FFC39430400CEFD394395006EF242B
:101A4E00D0FF801A900002120E95FFC39461400CD5
:101A5E00EFD394665006EF24A9FF80027F00EF7546
:101A6E00F010A4FFE5F04CFEEF4DFF900003120EB8
:101A7E0095FDC39430400CEDD394395006ED24D02F
:101A8E00FD80259001A0E0FBA3E0FAA3E0F9900011
:101A9E0003120E95FDC39461400CEDD3946650066F
:0B1AAE00ED24A9FD80027D00EF4DFF3C
:011AB900220A
:10154700E47880F6122AB3C286E4F5A775E101F5BF
:10155700E275E34043C91090019EF0A3F090019F0C
:10156700E004F0700690019EE004F090019EE070A8
:1015770004A3E0640E70E643B28FE4F5A9122A4A89
:10158700E4FF122A0B43EF04E490019EF0A3F090CE
:10159700019EE0FEA3E0FFC39401EE940050157D89
:1015A7000112299390019FE004F070E390019EE0FF
:1015B70004F080DBE4F520C20AC208C20EC20DC2E5
:1015C7000C7880F608F67826F618F6782CF690014F
:1015D7009EF0A3F090019EE0FEA3E0FFC3EE94010E
:1015E700501C74002FF58274003EF583E4F09001DF
:1015F7009FE004F070DE90019EE004F080D6E49056
:10160700019EF0A3F090019EE0FEA3E0FFC394408B
:10161700EE9400501C74002FF58274013EF583E4AC
:10162700F090019FE004F070DC90019EE004F080F0
:10163700D4122AE9E4F5A7E5EF20E10CE5EF540819
:10164700D394004003D38001C392037D08E4FF12C3
:1016570029C3E4782BF67823F6900183E0FBA3E017
:10166700FAA3E0F97823E6FF75F010A4F58285F078
:1016770083120E95FE782B26F6EE600578230680FA
:10168700D8EFD394004035900183E0FBA3E0FAA3A1
:10169700E0F990000D12106F120E7CFF7455120EB8
:1016A700C2120E7C64556002D20C74AA120EC212CA
:1016B7000E7C64AA6002D20CEF120EC2E5EF540250
:1016C700D3940040047F018002E4FF121840900188
:1016D7009DEFF090019DE020E03CC20974FF782E59
:1016E700F608F608F608F67E007F107D007B007A84
:1016F7000079341210F69001A374FFF0A3741BF065
:10170700A374DDF0A3E4F0A37410F07B007A0079F2
:10171700341226D38002D20912197E7832A606081F
:10172700A60790019DE030E103021808E4A3F0A3A7
:10173700F090019FE0C4F8540FC868FF90019EE045
:10174700C454F048FE900183E0FBA3E0FAA3E0F95C
:101757008F828E83120E9570030217FFE92FF9EA25
:101767003EFA900004120E9520E27CE490019CF072
:1017770090019CE0FDC3781A96506C90019FE0C4DD
:10178700F8540FC868FF90019EE0C454F048FE90DB
:101797000183E0FBA3E0FAA3E0F98F828E83120EA8
:1017A70095FF7E00C006C0077C0090019FE0C4F84B
:1017B700540FC868FF90019EE0C454F048FEE92F1B
:1017C700F9EA3EFA90000D12106F782BE68DF0A41F
:1017D70029F9EA35F0FA7D00D007D0061210F69005
:1017E700019CE004F0808990019FE004F07006906E
:1017F700019EE004F00217387F01122A95C20B8080
:1018070007E4FF122A95D20BE490019EF0A3F09013
:10181700019EE0FEA3E0FFC39401EE940050197A05
:10182700007B967D031224EE90019FE004F070DFA9
:0818370090019EE004F080D74F
:01183F002286
:052AE400782CE6FF2242
:03002300021ABA04
:101ABA00C0E0C0F0C083C082C0D075D000C000C0F2
:101ACA0001C002C003C004C005C006C00730994463
:101ADA00C2997826067926E77881667018F67826FC
:011AEA00F605
:101AEB00900186740AF000900186E014F0E070F625
:041AFB00C286801F00
:101AFF009001867414F000900186E014F0E070F607
:101B0F007826E62400F582E43401F583E0F5992088
:101B1F009803021BC2209A08200A05C298021BBE16
:101B2F00C29A7825E6062400F582E43400F583E5B1
:101B3F0099F0C298E6FFB40112900000E0FE700326
:101B4F00F68070EE54072402782DF6EFB4020D786C
:101B5F002DE6B40907900001E02403F67825E6FF8F
:101B6F00FD7C00B40007ECB40103F68046EFC378A8
:101B7F002D96403FED24FFFDEC34FFFC7B017A00F6
:101B8F00790012216B7825E624FFF582E434FFF506
:091B9F0083E06F60047600801AF7
:101BA8009001867414F000900186E014F0E070F65D
:101BB800782A0612002678257600D007D006D005A8
:101BC800D004D003D002D001D000D0D0D082D083AE
:051BD800D0F0D0E03266
:052AE900782AE6FF223F
:10221B00900001E075F010A4FF900183E0FBA3E0B8
:10222B00FAA3E02FF9EA35F0FA90000D12106F9037
:10223B000189782CE6FF18E68FF0A4FFE02FF582DA
:0F224B00E435F0F583120E95FF7B017A01798758
:10225A00900196EFF0A3EBF0A3EAF0A3E9F0900166
:10226A0097E0FBA3E0FAA3E0F9EA494B6022900168
:10227A0097A3A3120E7CFF900196E0FD7C00122A20
:10228A00A4900197E0FBA3E0FAA3E0F9EF120EC2D3
:10229A0090019A7414F00090019AE014F0E070F63C
:1022AA00900196E0F5997F0112295E3099FDC29955
:0122BA002201
:10273B009001007478F07825E624FFF582E434FFED
:09274B00F583E0900101F07F022A
:1027540090FFFF1210C5EFF090FFFF1210C585081F
:0B27640083850982A3E07881F6D2860D
:10276F008508838509827414F0850883850982E0C2
:0B277F00D39400400600E014F080EE50
:0C278A00900100E0F5999000020210C5DB
:10279600C9EFC9E964017028EDC39B403E781AE68B
:1027A600FFEB2FFFE433FEEDC39FEE6480F87480E9
:1027B600985028D20AC3ED9B782CF678277601220A
:1027C600CFE9CFEFB4021ACFEBCFCEEDCEEE6F70DE
:1027D6000AD20A782CF67827760222C20AE47827EB
:0227E600F622D9
:1023DD00900196ECF0A3EDF0C9EFC9BAFF19BBFF60
:1023ED0016900196E06A7003A3E06B7067D20A78CD
:1023FD002CF67827E9F622E964017035C390019730
:10240D00E09B900196E09A4026781AE62BFFE43A7D
:10241D00FEE0FCA3E0FDC39FEC9E5013D20ACFEB70
:10242D00CFCEEDCEC3EE9F782CF6782776012280A5
:10243D0023CFE9CFEFB40222CEEACECFEBCF90017E
:10244D0096E06E7003A3E06F700AD20A782CF678CE
:0B245D0027760222C20AE47827F6224C
:10002600900000E0FE54F8900188F0EE12109F0058
:100036007209007F0A009210009B1100AC1200C3E7
:100046001900D91A00FE2001042801982902D93383
:10005600031437035039036A41037549038050037B
:10006600D46102A37003CC9800000404900001E060
:10007600FD782FE6FB7F018027900001E0FCA3E0DE
:10008600FD782EE6FA08E6FB7F01802BD20A782758
:100096007603020404900001E0FD7831E6FB7F025E
:1000A600122796020404900001E0FCA3E0FD7830DC
:1000B600E6FA08E6FB7F021223DD02040490000143
:1000C600E0FD782FE6FB7F01122796200A03020443
:1000D60004801A900001E0FCA3E0FD782EE6FA0801
:1000E600E6FB7F011223DD200A03020404900100CF
:1000F6007478F07F0102040175EF10020404C2ACAB
:10010600E4900187F0D2867B017A0179877F7F129E
:10011600225A7B017A0179877F1812225A7B017A4B
:100126000179877F0512225A7823E6122253782E08
:10013600E6122253782FE61222537830E612225323
:100146007831E61222537832E61222537833E612D9
:100156002253E4900189F0900189E0FFC394105086
:100166001074342FF8E6122253900189E004F080CF
:0F017600E6900187E0FF7B007A00790012225AA1
:10018500900195740AF000900195E014F0E070F686
:1001950002028E900001E0FFC3782396400302021D
:1001A50095EF75F010A4FF900183E0FBA3E0FAA39F
:1001B500E02FF9EA35F0FA900192EBF0A3EAF0A30B
:1001C500E9F0C2ACE4900187F0D2867B017A01792F
:1001D500877F7F12225A7B017A0179877F0D122250
:1001E5005A900192E0FBA3E0FAA3E0F9120E7C120B
:1001F5002253900192E0FBA3E0FAA3E0F9900001FD
:10020500122250900192E0FBA3E0FAA3E0F99000DE
:1002150002122250900192E0FBA3E0FAA3E0F990CC
:100225000003122250900192E0FBA3E0FAA3E0F94B
:10023500900004122250E4900189F0900189E0FFBA
:10024500C394085026900192E0FBA3E0FAA3E024B2
:1002550005F9E43AFA7E00E92FF9EE3AFA120E7C36
:10026500122253900189E004F080D0900187E0FFCD
:090275007B007A00790012225A84
:10027E00900195740AF000900195E014F0E070F68C
:10028E00C286D2AC0204049001007478F0E4A3F0AC
:10029E007F02020401122ADA784412100D90010036
:1002AE00747CF07844E6A3F008E6A3F008E6A3F029
:1002BE0008E6A3F07C007D057B017A01790012210E
:1002CE006B900105EFF07F06020401900001E0FF44
:1002DE00B4010FA3E0FDA3E0782ECDF608EDF602F3
:1002EE0003CCEFB4020A900002E0782EF60203CCA3
:1002FE00900001E0B4030CA3E0FFA3E07830CFF64A
:10030E0008EFF60203CCE4900189F0900189E0FF3A
:10031E00C394105027900001E0FEEFC39E501D9035
:10032E000189E02402F582E43400F583E0FE7434A2
:10033E002FF8EEF6900189E004F080CFE47843F6D2
:10034E00807C7A007B327D01782CE6FF1224EE90C1
:10035E000001E0FDE4FF1229C3020404900001E055
:10036E0024FF9202020404900001E024FF92010295
:10037E000404782CE6600890018B7402F0800E90D5
:10038E00018B200D057403F080037401F0900100C1
:10039E007479F090018BE0900101F07C007D027B7E
:1003AE00017A01790012216B900102EFF07F0312A6
:1003BE00275490018BE06401703CD20E8002D2086B
:1003CE00788076F180307A007B327D017F001224B6
:1003DE00EE9001007479F0900001E0900101F07C44
:1003EE00007D027B017A01790012216B900102EFF0
:1003FE00F07F03122754900188E064A06003020688
:10040E0098781AE6B4010B7A007B327D017F0112D7
:10041E0024EE900000E064A1600302054BA3E0C34C
:10042E007823964003020540900183E0FBA3E0FA97
:10043E00A3E0F9900001E0FF75F010A4F58285F0BD
:10044E0083120E9590018BF0EF75F010A4FFE92F3B
:10045E00F9EA35F0FA900004120E9530E23C900065
:10046E0001E0FF12000390018BEFF0900100747F0A
:10047E00F0A3EFF02402FDE433FC7B017A01790056
:10048E0012216B90018BE0FE2402F582E43401F51B
:10049E0083EFF0EE2403FF020695900001E0FF12B9
:1004AE000003C2ACE4900187F0D28690018BE0D3BA
:1004BE00940640377B017A0179877F7F12225A900A
:1004CE00018BE0122253E4900189F090018BE0FF42
:1004DE00900189E0C39F500B12221B900189E0040A
:1004EE00F080E890018BE004F0802690018BE024F0
:1004FE0078122253E4900189F090018BE0FF900175
:10050E0089E0C39F500B12221B900189E004F080FA
:0F051E00E8900187E0FF7B007A00790012225AF3
:10052D00900195740AF000900195E014F0E070F6DA
:10053D000206879001007478F07F01020695900005
:10054D0000E064A260030206987823E6FFA3E0FEB4
:10055D00C39F400302068DA3E0FDC39F4003020627
:10056D008DEE9D400302068D900001E0900189F013
:10057D00E4900190F0A3F0900002E0FE900189E07C
:10058D00FFD39E5034120003900183E0FBA3E0FAE9
:10059D00A3E0F9900189E075F010A4F58285F08350
:1005AD00120E95FF900191E02FF0900190E0340034
:1005BD00F0900189E004F080BEC2ACE4900187F0B8
:1005CD00D2867B017A0179877F7F12225A90019022
:1005DD00E0FEA3E0FFC39480EE94005002800F90E4
:1005ED000190E04480122253900190A3E0FF12226B
:1005FD0054900001E0900189F0900002E0FF90011D
:10060D0089E0D39F5056E4A3F0900183E0FBA3E073
:10061D00FAA3E0F9900189E0FF75F010A4F5828549
:10062D00F083120E95FE90018AE0C39E5026EF7561
:10063D00F010A4FF900183A3A3E02FF9EA35F0FA9F
:10064D0090000D12106F90018A12223D90018AE0E8
:10065D0004F080B5900189E004F0809D900187E061
:0A066D00FF7B007A00790012225A88
:10067700900195740AF000900195E014F0E070F68F
:10068700C286D2AC800B9001007478F07F011227EC
:1006970054900188E064587057FA7B327D01782CBA
:1006A700E6FF1224EE9001997401F0A37401F0A300
:1006B7007401F07B017A00790112283990018BEFE0
:1006C700F0E0FE2478900100F0EE2401FDE433FC15
:1006D7007B017A01790012216B90018BE0FE2401E6
:1006E700F582E43401F583EFF0EE2402FF1227547C
:1006F700900188E0FF64806008EF64886003020966
:10070700057827E6B4010F7A007B327D01782CE665
:10071700FF1224EE8021E4900189F0900189E0FF27
:10072700C3781A9650117A007B327D011224EE901D
:100737000189E004F080E4900000E05407FF900195
:100747008BF0BF071390018A7401F0900001E090CD
:10075700018BF09000028008E490018AF09000017C
:10076700E090018CF090018BE014F0A3E0FFC378D8
:1007770023964003020905900183E0FBA3E0FAA357
:10078700E0F975F010EFA4F58285F083120E95FF5E
:1007970090018BE0D39F4002EFF07827E6B4010D7C
:1007A700782CE690018FF090018EF0800BE4900199
:1007B7008EF0781AE614A3F090018EE0782CF6906C
:1007C700018FE0FF782CE6D39F40030208F4E49002
:1007D7000189F090018BE0FF900189E0C39F4003FE
:1007E7000208E690018CE075F010A4FF900183E009
:1007F700FBA3E0FAA3E02FF9EA35F0FA9000041220
:100807000E9530E2030208DD900001120E95643860
:10081700705090018BE0D39404900189E0FF401160
:10082700A3E02F2402F582E43400F583E0FD0208FB
:10083700BD7825E6C39FFFE49400FE74FE2FF58282
:1008470074FF3EF583E0FD90018CE075F010A4FF86
:10085700900183E0FBA3E0FAA3E02FF9EA35F0FA71
:100867008054900183E0FBA3E0FAA3E0F990018CA8
:10087700E075F010A4F58285F083120E95FF7825B8
:10088700E6C39FFFE49400FE900189E07C002FFF00
:10089700EC3EFEA3E02FFFEC3EFE74FF2FF58274C3
:1008A700FF3EF583E0FD90018CE075F010A4FFE9B1
:1008B7002FF9EA35F0FA90000D12106F782CE6FF49
:1008C70018E68FF0A4FF900189E02FF582E435F058
:1008D700F583ED120ED4900189E004F00207DA9057
:1008E700018CE0FF122AC2782C060207C690018EFF
:1008F700E0782CF6900188E0B4880312273B90013A
:1009070088E064A86003020AA57827E6B4010F7A95
:10091700007B327D01782CE6FF1224EE8021E490E3
:100927000189F0900189E0FFC3781A9650117A0087
:100937007B327D011224EE900189E004F080E4907F
:100947000001E030E718547FFEA3E0FDEDFF9001C2
:1009570090EEF0A3EFF090018A7403F080139000FB
:1009670001E0FF900190E4F0A3EFF090018A740298
:10097700F090018AE0FF2400F582E43400F583E07B
:10098700FE74012FF582E43400F583E090018DF0C9
:10099700CFEECF90018CEFF090018DE0FF90018CAE
:1009A700E0FED39F4003020AA2EEC37823964003DA
:1009B700020A99900183E0FBA3E0FAA3E0F975F03E
:1009C70010EEA4F58285F083120E9590018BF078D6
:1009D70027E6B4010D782CE690018FF090018EF098
:1009E700800BE490018EF0781AE614A3F090018E44
:1009F700E0782CF690018FE0FF782CE6D39F400338
:100A0700020A87E4900189F090018BE0FF90018949
:100A1700E0C39F505D90018CE075F010A4FF90013A
:100A270083E0FBA3E0FAA3E02FF9EA35F0FA9000A0
:100A370004120E9520E233900189E0FFA3E02F24F2
:100A470002F582E43400F583E0FD90000D12106F8B
:100A5700782CE6FF18E68FF0A4FF900189E02FF5C8
:100A670082E435F0F583ED120ED4900189E004F0AD
:100A7700809690018CE0FF122AC2782C060209FBAF
:100A870090018EE0782CF690018BE0FF90018AE0D0
:0E0A97002FF090018CE004F002099F12273B23
:010AA500222E
:10F000007880E664F1600302F6B3784EF608F6788D
:04F0100081E6602114
:10F0140090019C740AF00090019CE014F0E070F6FA
:10F02400784F06E618700106784EB627DE08B6104B
:10F03400DAC2AFE4784AF618F6209833E4784EF64C
:10F0440008F6209826C3784FE6948818E69413505F
:01F054001AA1
:10F0550090019C740AF00090019CE014F0E070F6B9
:10F06500784F06E61870DA0680D7B29680CA7849D6
:10F07500A699C298E6FF641A6008EF640A60030265
:10F08500F16DE4784EF608F6209826C3784FE6949D
:07F095008818E69413501ADD
:10F09C0090019C740AF00090019CE014F0E070F672
:10F0AC00784F06E61870DA0680D7309884784AA62E
:10F0BC0099C298E4784EF608F6209826C3784FE665
:08F0CC00948818E69413501A11
:10F0D40090019C740AF00090019CE014F0E070F63A
:10F0E400784F06E61870DA0680D720980302F03DC0
:10F0F400784AA699C298E4784EF608F6209826C372
:0BF10400784FE6948818E69413501A28
:10F10F0090019C740AF00090019CE014F0E070F6FE
:10F11F00784F06E61870DA0680D720980302F03D84
:10F12F00784AA699C29818E6641A600302F6A4D228
:03F13F0086C299EC
:10F1420090019C7414F00090019CE014F0E070F6C1
:06F152007599783099FD6B
:10F1580090019C740AF00090019CE014F0E070F6B5
:10F16800C28602F6A47849E6FF6450600302F211F1
:10F17800784EF608F6209826C3784FE6948818E665
:04F188009413501A72
:10F18C0090019C740AF00090019CE014F0E070F681
:10F19C00784F06E61870DA0680D720980302F03D07
:0AF1AC00784AA699C298D286C2994B
:10F1B60090019C7414F00090019CE014F0E070F64D
:08F1C6007599793099FDC29999
:10F1CE0090019C7414F00090019CE014F0E070F635
:08F1DE007599013099FDC299F9
:10F1E60090019C7414F00090019CE014F0E070F61D
:06F1F600E4F5993099FDDB
:10F1FC0090019C740AF00090019CE014F0E070F611
:0EF20C00C28602F6A4EF64017047D286C29952
:10F21A0090019C7414F00090019CE014F0E070F6E8
:08F22A007599783099FDC29935
:10F2320090019C7414F00090019CE014F0E070F6D0
:06F24200E4F5993099FD8E
:10F2480090019C740AF00090019CE014F0E070F6C4
:10F25800C28602F6A47849E66402600302F33578B0
:10F268004EF608F6209826C3784FE6948818E69458
:03F2780013501A16
:10F27B0090019C740AF00090019CE014F0E070F691
:10F28B00784F06E61870DA0680D720980302F03D17
:10F29B00784AA699C298E408F618E6FF13B392963B
:10F2AB00EF25E0FECC74F0CCCD7400CDC3E49DEE25
:10F2BB009C502AE67F0025E0FEC39460501FE4F5C6
:10F2CB00A7758F037850EEF608EFF675B7A5788023
:10F2DB00E6F5B78F828E83E4F0F58F8004784B765A
:05F2EB00FFD286C2996C
:10F2F00090019C7414F00090019CE014F0E070F612
:08F300007599783099FDC2995E
:10F3080090019C7414F00090019CE014F0E070F6F9
:08F31800784BE6F5993099FDF0
:10F3200090019C740AF00090019CE014F0E070F6EB
:10F33000C28602F6A47849E66403600302F4947876
:10F340004EF608F6209826C3784FE6948818E6947F
:03F3500013501A3D
:10F3530090019C740AF00090019CE014F0E070F6B8
:10F36300784F06E61870DA0680D720980302F03D3E
:10F37300784AA699C298E4784EF608F6209826C3F0
:0BF38300784FE6948818E69413501AA7
:10F38E0090019C740AF00090019CE014F0E070F67D
:10F39E00784F06E61870DA0680D720980302F03D03
:10F3AE00784CA699C298784AE6FF139296EF25E01C
:10F3BE00FECC74F0CCCD7400CDC3E49DEE9C400326
:10F3CE0002F03DE67D0025E0FCC39460400302F0B0
:10F3DE003DE4F5A7758F01784CE675F020A42DFF5E
:10F3EE00E5F03C7850F608EFF6E4784DF6784DE609
:10F3FE00C394205047E408F608F6209816C3784FB9
:10F40E00E6948818E69413500A000806E61870EA87
:10F41E000680E720980302F03D75B7A57880E6F5E3
:10F42E00B778500806E618CEE6CE70010614F582BF
:10F43E008E83E599F0C298784D0680B1E4F58FD2AF
:03F44E0086C299DA
:10F4510090019C7414F00090019CE014F0E070F6AF
:08F461007599783099FDC299FC
:10F4690090019C7414F00090019CE014F0E070F697
:06F47900E4F5993099FD55
:10F47F0090019C740AF00090019CE014F0E070F68B
:10F48F00C28602F6A47849E6FD6404600302F55DC6
:10F49F00784EF608F6209826C3784FE6948818E63B
:04F4AF009413501A48
:10F4B30090019C740AF00090019CE014F0E070F657
:10F4C300784F06E61870DA0680D720980302F03DDD
:10F4D300784AA699C298E625E07852F608E4F678C9
:10F4E3004BF6784EF608F678520806E618CEE6CEC6
:10F4F30070010614F5828E83E493784B26F6784FD9
:10F5030006E618700106784FE6700418E664027088
:05F51300D6D286C2996A
:10F5180090019C7414F00090019CE014F0E070F6E7
:08F528007599783099FDC29934
:10F5300090019C7414F00090019CE014F0E070F6CF
:08F54000784BE6F5993099FDC6
:10F5480090019C740AF00090019CE014F0E070F6C1
:10F55800C28602F6A4ED6405600302F69B784EF6B7
:10F5680008F6209826C3784FE6948818E694135036
:01F578001A78
:10F5790090019C740AF00090019CE014F0E070F690
:10F58900784F06E61870DA0680D720980302F03D16
:10F59900784AA699C298E4784EF608F6209826C3C8
:0BF5A900784FE6948818E69413501A7F
:10F5B40090019C740AF00090019CE014F0E070F655
:10F5C400784F06E61870DA0680D720980302F03DDB
:0AF5D400784CA699C298D286C2991D
:10F5DE0090019C7414F00090019CE014F0E070F621
:08F5EE0075997F3099FDC29967
:10F5F60090019C7414F00090019CE014F0E070F609
:10F606007599203099FD784AE625E0FC784CE67538
:10F61600F020A42400FFE5F03C7852F608EFF6E46B
:08F62600784BF6784DF6C2990D
:10F62E0090019C7414F00090019CE014F0E070F6D0
:10F63E007852E6FE08E6F5828E83E493F5993099CA
:10F64E00FD78520806E618CEE6CE70010614F58255
:10F65E008E83E493784B26F6784D06E6B420BFC22F
:01F66E009902
:10F66F0090019C7414F00090019CE014F0E070F68F
:08F67F00784BE6F5993099FD86
:10F6870090019C740AF00090019CE014F0E070F681
:10F69700C28680097849E6B4060375EF107849E613
:0CF6A7006407600302F03D7880F6D2AFEB
:01F6B3002234
:102665007F0012295E20090B7A007B327D017F00F5
:102675001224EE300C0B7A007B1E7D017F001224A4
:10268500EE300817300D147A007B327D01782CE688
:10269500FF1224EEC208121FCFD209200B0C300DF9
:1026A50009788076F1121FCFD20B300E0B300D0852
:1026B500C20E122AB312F000200D12122AD0E47BAA
:0E26C5002C7A01F9F8C3120FC95002D20D226F
:102A2C0075EF027F64DFFE121547122AE4122A6644
:0E2A3C00E4FFFE12291F122665122AEE80F812
:101CF600005EBCE2613FDD83C29C7E20A3FD1F41E6
:101D06009DC3217FFCA2401E5F01E3BD3E6082DCD5
:101D1600237D9FC1421CFEA0E1BF5D0380DE3C62C5
:101D2600BEE0025CDF81633D7C22C09E1D43A1FFB5
:101D36004618FAA427799BC584DA3866E5BB5907A5
:101D4600DB856739BAE406581947A5FB7826C49A95
:101D5600653BD987045AB8E6A7F91B45C6987A2485
:101D6600F8A6441A99C7257B3A6486D85B05E7B975
:101D76008CD2306EEDB3510F4E10F2AC2F7193CD65
:101D8600114FADF3702ECC92D38D6F31B2EC0E5055
:101D9600AFF1134DCE90722C6D33D18F0C52B0EE45
:101DA600326C8ED0530DEFB1F0AE4C1291CF2D7335
:101DB600CA947628ABF517490856B4EA6937D58B25
:101DC6005709EBB536688AD495CB2977F4AA481615
:101DD600E9B7550B88D6346A2B7597C94A14F6A805
:101DE600742AC896154BA9F7B6E80A54D7896B35F5
:0A1DF6000000000000002B96B9DD8C
:032A9100010F0A28
:102A660090019C12103EFFFFFFFF90019CE0FCA32B
:082A7600E0FDA3E0FEA3E0FF78
:012A7E002235
:10216B0090FFFE1210C5ECF0A3EDF090FFFD1210E6
:0F217B00C5EBF0A3EAF0A3E9F090FFFC1210C54A
:10218A00850883850982A3A3E4F0850883850982EB
:10219A00F0A3F09000071210E9E0FEA3E0FF850823
:1021AA0083850982E0FCA3E0FDC39FEE6480F8EC1E
:1021BA00648098504C9000041210E9E0FBA3E0FA06
:1021CA00A3E0F98D828C83120E95FF850883850919
:1021DA0082A3A3E06FFF9000031210E9EFF09000D2
:1021EA00031210E9E0901CF693850883850982A3FF
:1021FA00A3F0850883850982E475F001120F2C800B
:0B220A0092850883850982A3A3E0FFF2
:062215009000090210C553
:0E2AA400CEEDCEEE6F7848F6E6901CF693FF6E
:012AB2002201
:1029C300EF7020F5A77598D0E589540F4420F58959
:1029D300438E08CFEDCFEF901DF593F58DD28ED2B8
:0529E300ACC2BCD2AF44
:0129E80022CC
:1027E800781212102500000000781612102500003B
:1027F8000000780A7664E47849F67849E6FFC394DD
:1028080001502DEF25E025E0240BF8E4F6EF25E054
:1028180025E0240CF8E4F6EF25E025E0240DF8E4A3
:10282800F6EF25E025E0240EF8E4F678490680CA9C
:01283800227D
:102A4A00D2AFD2A9C2BBE589540F4401F589758E6C
:0C2A5A0002758CECE4F58AD28C0227E8AF
:0620AC0090FFFF1210C5B9
:1020B200850883850982E4F0850883850982E0FF2B
:1020C200C394014003022165EF25E025E0240EF8C8
:1020D200E6FFD39400406EE025E025E0240CF8E60C
:1020E2007063EF30E013E0FF25E025E0240EF8E610
:1020F200D3940140047D01800A7D0085088385090F
:1021020082E0FF122889850883850982E0FF25E0A5
:1021120025E0240EF8E6B401057D00122889850821
:1021220083850982E0FF25E025E0240EF816E660AB
:1021320014EF25E025E0240DF8E6FEEF25E025E08A
:10214200240CF8EEF6850883850982E025E025E077
:10215200240CF8E6600116850883850982E004F004
:032162000220BA9E
:062165009000010210C50C
:03000B0002246864
:10246800C0E0C0F0C083C082C0D0E8C0E0E9C0E0EE
:10247800EAC0E0EBC0E0ECC0E0EDC0E0EEC0E0EFA9
:10248800C0E0758CEC7812121001EF2401FFE43ED5
:10249800FEE43DFDE43CFC781212100D780A16E6C5
:1024A800701B7816121001EF2401FFE43EFEE43D94
:1024B800FDE43CFC781612100D780A76641220AC04
:1024C8001229E9D0E0FFD0E0FED0E0FDD0E0FCD05A
:1024D800E0FBD0E0FAD0E0F9D0E0F8D0D0D082D05C
:0624E80083D0F0D0E032C9
:1029930090FFFF1210C5EDF090FFFF1210C5EFF08E
:1029A300850883850982E0FFC39401500DA3E0FEEF
:1029B300EF25E025E0240BF8EEF69000020210C5A7
:1024EE0090FFFE1210C5EAF0A3EBF090FFFF121062
:1024FE00C5EDF090FFFF1210C5EFF085088385093A
:10250E0082E0FFC394015056EF25E025E0240EF83B
:10251E00E6704BE0FB25E025E0240CF8E6703FA3C7
:10252E00E025E004FF850883850982E0FA25E02591
:10253E00E0240EF8EFF6850883850982A3A3E0FE5A
:10254E00A3E0FF7C007D0A120EF6EA25E025E024CA
:10255E000DF8EFF6EB25E025E0240CF8E4F69000FC
:04256E00040210C58E
:1028890090FFFF1210C5EDF090FFFF1210C5EFF099
:10289900850883850982E0FFC39401501EEF25E076
:1028A90025E0240BF8E66013A3E070047F018002A1
:1028B9007F00850883850982A3EFF0850883850950
:1028C90082E07006A3E024FF92969000020210C5F0
:092AD000C2AF7812121001D2AF5E
:012AD90022DA
:092ADA00C2AF7816121001D2AF50
:012AE30022D0
:10295E0090FFFF1210C5EFF0850883850982E070A5
:10296E00057810F608F6301016780FE675F064A4A8
:10297E00FFC37811E69F18E695F05003E4F5D39067
:05298E0000010210C56C
:102A0B00D210E47810F608F6EF780F6003F6800228
:102A1B00760AE4F5D975D2FF75D940F5D375EF0673
:012A2B002288
:0F2AB300C210E47810F608F6780F76FFF5D922F6
:1029E900781106E618700106301016780FE675F0B2
:1029F90064A4FFC37811E69F18E695F05003E4F547
:022A0900D322D6
:08291F0090019CEEF0A3EFF023
:10292700E4A3F0A3F090019CE0FEA3E0FFC39001B5
:102937009FE09F90019EE09E501C7FE87E0312253A
:10294700EC7F0112295E90019FE004F070D790019F
:062957009EE004F080CFB9
:01295D002257
:0825EC009001A7EEF0A3EFF04F
:1025F400D394FAEE940050199001A7A3E0FFEFD30F
:102604009400405C000000000000000000001F80F7
:10261400ED9001A7E0FFA3E09001AACFF0A3EFF0B3
:10262400D39001ABE094FA9001AAE0940040177FA4
:10263400FA7E001225EC9001ABE02406F09001AA8A
:10264400E034FFF080DAD39001A8E094009001A771
:10265400E09400400B9001AAE0FEA3E0FF1225ECF9
:012664002253
:1022BB009001AC7401F0A37401F0A374A6F07B0140
:0622CB007A0179A47D02F6
:0E22D1009001A8EBF0A3EAF0A3E9F0A3EDF072
:1022DF007F0112295E9001ACE0FBA3E0FAA3E0F9C5
:1022EF00120F422400FFE5F03460FE9001A8E0F9E0
:1022FF00A3E0FAA3E09001AFC9F0A3EAF0A3E9F0DD
:10230F00E4FD9001ABE0FCEDC39C5022EF2DF58274
:10231F00E43EF583E493FC9001AFE0FBA3E0FAA366
:10232F00E0F98D82758300EC120ED40D80D49001EC
:10233F00ABE0FFA3E0FBA3E0FAA3E0F9E48FF00228
:02234F000F6D10
:101EF00090019E7412F0A37434F09001A67401F066
:101F0000A37401F0A374A0F07B017A01799E7D0295
:0E1F10009001A2EBF0A3EAF0A3E9F0A3EDF03C
:101F1E007880E664F16003021FCE122AB3C2AFE4EA
:101F2E00F5A7758F01A3E0FBA3E0FAA3E0F9120F6A
:101F3E00422400FFE5F034607849F608EFF6900190
:101F4E00A2E0FBA3E0FAA3E0F9784DC6EBC608C603
:101F5E00EAC608C6E9C6E4784BF69001A5E0FF781C
:101F6E004BE6C39F503C784DCBE6CB080806E618EF
:101F7E00CAE6CA70010614F9120E7C784CF675B7D3
:101F8E00A57880E6F5B7784CE6FF78490806E6189E
:101F9E00CCE6CC70010614F5828C83EFF0784B06FC
:101FAE0080B8E4F58F9001A5E0FFA3E0FBA3E0FA73
:101FBE00A3E0F9E48FF0120F6DD2AFE4FF122A0BFB
:011FCE0022F0
:1028D9007880E664F1703EC2AF122AB3E4F5A775B9
:1028E9008F03784A766008F67849F675B7A5788037
:1028F900E6F5B7784AE6FE08E6F5828E83E4F02627
:10290900F618740236F61806E6B408DFE4F58FD235
:05291900AFFF122A0BC4
:01291E002296
:101FCF001228D9E49001A0F0A3F07B019001A604A0
:101FDF00F0A37401F0A374A0F01B7A00792E7D1684
:101FEF00121F10121EF0E490019DF090019DE0C3AE
:101FFF00781A9640030220A4E490019CF09001838C
:10200F00E0FBA3E0FAA3E0F990019CE0FF75F0106C
:10201F00A4F58285F083120E956071EF75F010A410
:10202F00FF900183A3A3E02FF9EA35F0FA90000D9A
:10203F0012106F90019DE0FF782BE68FF0A429F925
:10204F00EA35F0FAEBC0E0EAC0E0E9C0E0900183C6
:10205F00E0FBA3E0FAA3E0F990019CE075F010A477
:10206F00F58285F083120E95FD9001A67401F0A301
:10207F007401F0A374A0F0D0E0F9D0E0FAD0E0FB47
:10208F00121F1090019CE004F002200C90019DE0C3
:0C209F0004F0021FFA121EF0E47880F634
:0120AB002212
:051840009001A0EFF093
:10184500E49001A6F0A3F09001A3F07B019001AC18
:1018550004F0A37401F0A374A6F01B7A00792E7D21
:10186500161222D11222BB9001A4E0B4120CA3E0FF
:10187500B434079001A3E04401F0E49001A2F09094
:1018850001A2E0C3781A964003021962E49001A10F
:10189500F0900183E0FBA3E0FAA3E0F99001A1E059
:1018A500FF75F010A4F58285F083120E9570030282
:1018B50019599001A0E0606AEF75F010A4FF90013E
:1018C50083A3A3E02FF9EA35F0FA90000D12106F0B
:1018D5009001A2E0FF782BE68FF0A429F9EA35F014
:1018E500FAEBC0E0EAC0E0E9C0E0900183E0FBA3C9
:1018F500E0FAA3E0F99001A1E075F010A4F5828566
:10190500F083120E95FD9001AC7401F0A37401F003
:10191500A374A6F0D0E0F9D0E0FAD0E0FB1222D112
:101925008029900183E0FBA3E0FAA3E0F99001A1EF
:10193500E075F010A4F58285F083120E95FF9001F5
:10194500A7E02FF09001A6E03400F09001A1E0049B
:10195500F00218969001A2E004F00218841222BB4E
:101965009001A4E0B4120CA3E0B434079001A3E005
:081975004402F09001A3E0FF21
:01197D002247
:100AA600020E30E86480F8E933E83360110460F040
:100AB600ED33EC337009E8FCE9FDEAFEEBFF2204B6
:100AC60060DED3EB9FEA9EE99DE8C2E78CF0C2F7B1
:100AD60095F0400CE8CCF8E9CDF9EACEFAEBCFFB7D
:100AE600120DFB85D0F05804700320D5B3E80470CE
:100AF600075002B2D5020E3A92D5EC0460F7E4CC68
:100B0600C0E0C398F8603B94186008400DD0E0FB45
:100B1600020E12E4FBFAC9FC8028E830E406E4C9B8
:100B2600FBE4CAFCE830E305E4C9CACBFCE8540799
:100B36006010F8C3E913F9EA13FAEB13FBEC13FCA4
:100B4600D8F130F52FC3E49CFCEF9BFFEE9AFEED47
:100B560099FDD0E0FBEF4E4D4C701222DB03020EE6
:100B660037EC2CFCEF33FFEE33FEED33FDED30E7D3
:100B7600EB020E12EF2BFFEE3AFEED39FDD0E0FB55
:100B860050130BBB0003020E3AED13FDEE13FEEFFE
:080B960013FFEC13FC020E1228
:100B9E00EC4D6011E8497017ED33EC3304600DE451
:100BAE00FCFFFEFD22E933E8330470F8020E30122A
:100BBE000DFB58046009E4CC24815006285009022C
:100BCE000E3A284003020E37C0E0EB4A7044B9805B
:100BDE0006D0E0FB020E26EF4E701CBD8008EBFF28
:100BEE00EAFEE9FD80EBE98DF0A4FEE5F0020C874C
:100BFE00E9CDF9EAFEEBFFEF89F0A4FCE5F0CE8932
:100C0E00F0A42EFFE435F0CD89F0A42DFEE435F0EE
:100C1E008067EF4E7005BD80D780C3EF8BF0A4AC1C
:100C2E00F0EE8BF0A42CFCE435F0F8EF8AF0A42C57
:100C3E00E5F038FCE433CB8DF0A42CFCE5F03BF86A
:100C4E00EE8AF0A42CFCE5F038F8E433CF89F0A45A
:100C5E002CFCE5F038CF3400CE89F0A42FFFE5F060
:100C6E003EFEE433C98DF0A42EFEE5F039CD8AF0B8
:100C7E00A42FFFE5F03EFEE43DFD33D0E0FB500730
:100C8E000BBB000F020E3AEC2CFCEF33FFEE33FEE3
:060C9E00ED33FD020E1211
:100CA400020E3AEC5D046005E859047003020E304C
:100CB400120DFB580460F6EC4860F2EC7004FDFE83
:100CC400FF22C860DB2481C85009C3986002500623
:100CD400020E379850CAF582E9294B4A7005AB8257
:100CE400020E2675F0007C1A7880C3EF9BEE9AED15
:100CF40099400DC3EF9BFFEE9AFEED99FDE842F09B
:100D0400DC23ACF0D0E0FFD0E0FED0E0FDAB8220ED
:100D1400E7101BEB60BAEC2CFCEF33FFEE33FEED77
:100D240033FD020E12E803F830E705C0F075F00059
:100D3400EF2FFFEE33FEED33FD40B830E7C280AA5B
:100D440074F8CC6480CCC86480C8F58204604FC356
:100D5400EB9FF5F0EA9E42F0E99D42F0E89C45F0F5
:100D6400603C501DE5825FFFE582D313CB5BCBF47F
:100D74002B5582FB50280ABA002409B900200880A8
:100D84001DE5825BFBE582D313CF5FCFF4C3132F42
:100D94005582FF50090EBE00050DBD00010CC3EBCA
:100DA4009FF5F0EA9E42F0E99D42F0E89C45F06030
:090DB40007CC4820E701B3EC2252
:100DBD0075F020800E75F010800575F0087D007EB1
:100DCD00007F003392D530D503120FA5EC334010C0
:100DDD00EF33FFEE33FEED33FDEC33FCD5F0ED22BA
:0E0DED00E5F0247EA2D513CC92E7CDCEFF22F6
:101E00009001A712101974FFFFFEFDFC9001A7E0DE
:101E1000F8A3E0F9A3E0FAA3E0FBC3120FC960380E
:101E20007F807E967D187C4B9001A7E0F8A3E0F9B7
:101E3000A3E0FAA3E0FB120D446002501B7F807EFA
:101E4000967D187CCB9001A7E0F8A3E0F9A3E0FA17
:101E5000A3E0FB120D44500F9001A7E0FCA3E0FDAE
:101E6000A3E0FEA3E0FF229001A7E0FCA3E0FDA316
:101E7000E0FEA3E0FF120E459001AB121019900195
:101E8000ABE0FCA3E0FDA3E0FEA3E0FFEC120DBD80
:101E9000C8ECC8C9EDC9CAEECACBEFCB9001A7E028
:101EA000FCA3E0FDA3E0FEA3E0FF120AA9E4FBFA15
:101EB000F9F8120D44602640249001ABE0FCA3E049
:101EC000FDA3E0FEA3E0FFEF24FFFFEE34FFFEEDF5
:101ED00034FFFDEC34FFFC9001AB1210199001AB04
:101EE000E0FCA3E0FDA3E0FEA3E0FFEC120DBD22A9
:100DFB00E9D2E7C933E833F892D5EDD2E7CD33EC3E
:070E0B0033FC5002B2D522B6
:100E1200EC30E7100FBF000C0EBE00080DBD000441
:100E22000BEB6014A2D5EB13FCED92E7FD2274FFED
:100E3200FCFDFEFF22E480F8A2D574FF13FC7D8046
:030E4200E480EF5A
:100E4500EDD2E7CD33EC3392D524814006E4FFFEA5
:100E5500FDFC22FCE4CFCECDCC24E0501174FF8004
:100E6500EDC3CC13CCCD13CDCE13CECF13CF0470A1
:070E7500F030D5DE020FA5ED
:0300000002235187
:0C235100787FE4F6D8FD758181022398A6
:100E7C00BB010689828A83E0225002E722BBFE0274
:090E8C00E32289828A83E49322A7
:100E9500BB010CE58229F582E5833AF583E0225012
:100EA50006E92582F8E622BBFE06E92582F8E2225C
:0D0EB500E58229F582E5833AF583E4932276
:100EC200BB010689828A83F0225002F722BBFE010F
:020ED200F32209
:100ED400F8BB010DE58229F582E5833AF583E8F054
:100EE400225006E92582C8F622BBFE05E92582C800
:020EF400F222E8
:100EF600C2D5EC30E709B2D5E4C39DFDE49CFCEE17
:100F060030E715B2D5E4C39FFFE49EFE121122C35B
:100F1600E49DFDE49CFC800312112230D507C3E456
:060F26009FFFE49EFE2285
:100F2C00C5F0F8A3E028F0C5F0F8E5821582700250
:060F3C001583E038F022ED
:100F4200BB010A89828A83E0F5F0A3E0225006877A
:100F5200F009E71922BBFE07E3F5F009E31922893C
:0B0F6200828A83E493F5F0740193226F
:100F6D00BB010789828A83020F2C500B09C5F0271C
:100F7D00F7C5F01937F722BBFE0D09F8E325F0F39D
:100F8D00C5F019E338F322F889828A837401932519
:080F9D00F0C5F0F8E4933822DE
:0E0FA500C3E49FFFE49EFEE49DFDE49CFC225D
:100FB300EB9FF5F0EA9E42F0E99D42F0EC6480C8B5
:060FC30064809845F02255
:100FC900EB9FF5F0EA9E42F0E99D42F0E89C45F07E
:010FD90022F5
:100FDA00E86010ECA2E713FCED13FDEE13FEEF132D
:040FEA00FFD8F0221A
:100FEE00E8600FEFC333FFEE33FEED33FDEC33FC61
:030FFE00D8F12205
:0C100100E6FC08E6FD08E6FE08E6FF221B
:0C100D00ECF608EDF608EEF608EFF6220F
:0C101900ECF0A3EDF0A3EEF0A3EFF0224A
:10102500D083D082E493F608740193F60874029392
:09103500F608740393F6740473C9
:10103E00A8828583F0D083D08212105512105512DB
:10104E001055121055E473E493A3C583C5F0C58300
:10105E00C8C582C8F0A3C583C5F0C583C8C582C8FC
:01106E00225F
:10106F00BB010DE58229F582E5833AF583021196DE
:10107F005007E92582F802118DBBFE07E92582F89A
:10108F0002119FE58229F582E5833AF5830211A8C3
:10109F00D083D082F8E4937012740193700DA3A3E0
:1010AF0093F8740193F5828883E4737402936860F4
:0610BF00EFA3A3A380DFF4
:1010C500E5092582F582E5083583F583B5080485AC
:1010D50082092210AF06858209F50822858209F565
:0410E50008D2AF225C
:0D10E900E5092582F582E5083583F58322AF
:1026D3009001A0EBF0A3EAF0A3E9F0E49001A8F0E5
:1026E300A3F09001A674FFF5F012117745F0603C5A
:1026F3009001A3E0FBA3E0FAA3E0F9120E7CFF90A4
:1027030001A0E0FBA3E0FAA3E0F99001A8E475F0CF
:102713000112117785F082F583EF120ED4EF60C2B8
:102723009001A4E475F001120F2C80B69001A0E093
:08273300FBA3E0FAA3E0F92288
:102572009001A3EBF0A3EAF0A3E9F0A3EBF0A3EA46
:10258200F0A3E9F09001A6E0FBA3E0FAA3E0F912C0
:102592000E7C600C9001A7E475F001120F2C80E410
:1025A2009001A6E0FBA3E0FAA3E0F9120E7C6D70A5
:1025B20001229001A3E0FBA3E0FAA3E0F9EBC0E063
:1025C200EAC0E0E9C0E0A3E0FBA374FFF5F012115A
:1025D20077FAD082D083D0E06B7009E5F065827023
:0A25E20003EA658370BAFBFAF922E0
:1010F600EF4E6012EF60010EEDBB010B89828A8311
:10110600F0A3DFFCDEFA2289F05007F709DFFCA91D
:0C111600F022BBFEFCF309DFFCA9F02274
:10235D00022A2CE493A3F8E493A34003F68001F240
:10236D0008DFF48029E493A3F85407240CC8C33381
:10237D00C4540F4420C8834004F456800146F6DF50
:10238D00E4800B0102040810204080902A7FE47E37
:10239D00019360BCA3FF543F30E509541FFEE49345
:1023AD00A360010ECF54C025E060A840B8E493A30C
:1023BD00FAE493A3F8E493A3C8C582C8CAC583CA37
:1023CD00F0A3C8C582C8CAC583CADFE9DEE780BEEF
:012A94000041
:10112200BC000BBE0029EF8DF084FFADF022E4CCB1
:10113200F875F008EF2FFFEE33FEEC33FCEE9DEC7A
:10114200984005FCEE9DFE0FD5F0E9E4CEFD22EDC0
:10115200F8F5F0EE8420D21CFEADF075F008EF2F0A
:10116200FFED33FD4007985006D5F0F222C398FDFB
:051172000FD5F0EA2298
:10117700A3F8E0C5F025F0F0E5821582700215832B
:06118700E0C838F0E82288
:09118D00E6FB08E6FA08E6F92287
:09119600E0FBA3E0FAA3E0F9225A
:09119F00E2FB08E2FA08E2F92281
:0C11A800E493FB740193FA740293F922A3
:00000001FF
